:100000000428FF3FFF3FFF3F031383129F01831626
:100010008501860187018801890183128501860196
:10002000870188018901FF30A0008130A100BD3027
:10003000A200A530A300A530A400BD30A5008130EA
:10004000A600FF30A700200886000130880002309B
:10005000FB00FF30FA00FB0B2E283128FA0B2E286C
:100060002B284A30FA00FA0B332821088600023088
:1000700088000230FB00FF30FA00FB0B40284328C9
:10008000FA0B40283D284A30FA00FA0B452822088E
:100090008600043088000230FB00FF30FA00FB0BC2
:1000A00052285528FA0B52284F284A30FA00FA0BEA
:1000B000572823088600083088000230FB00FF30F4
:1000C000FA00FB0B64286728FA0B642861284A3081
:1000D000FA00FA0B692824088600103088000230E4
:1000E000FB00FF30FA00FB0B76287928FA0B762804
:1000F00073284A30FA00FA0B7B2825088600203046
:1001000088000230FB00FF30FA00FB0B88288B28A8
:10011000FA0B882885284A30FA00FA0B8D28260821
:100120008600403088000230FB00FF30FA00FB0BF5
:100130009A289D28FA0B9A2897284A30FA00FA0B39
:100140009F2827088600803088000230FB00FF309F
:10015000FA00FB0BAC28AF28FA0BAC28A9284A30D0
:10016000FA00FA0BB1282328B428FF3FFF3FFF3FD6
:02400E003A3F37
:00000001FF
